:1000000036C060C027C1E8C0E5C05CC05BC05AC054
:1000100059C058C057C056C0E3C054C053C00407AD
:1000200014233764A0FFFFFFFFFFFFFFFFFFFFFF69
:10003000FF000000000000000000000000000000C1
:1000400023456C98C9FF040714233764A0FFFFFF02
:10005000FFFFFFFFFFFFFFFFFF00000000000000A9
:10006000000023405F7AB4FFFFFFFFFFFF00112471
:100070001FBECFE5D2E0DEBFCDBF20E0A0E6B0E0FE
:1000800001C01D92A938B207E1F7E2E6F0E085E58C
:10009000808781E083831482128286831182AEE698
:1000A000B0E08EEF15968C9315978DEF17968C9385
:1000B0008BE0828788E58387612C712C88248A9461
:1000C00090D01AC19DCF989A1EBC1BBC19BC18BCFD
:1000D000089525B7277E25BF21E02FBD019728F081
:1000E00020E288952150E9F7F9CF089588EE93E052
:1000F000F0CF8CE287B986EC86B9369A3699FECF76
:100100008FEF809360000895369A3699FECF95B1AF
:100110008091600089270895811101C0D4CF81505A
:1001200090E0FC01E25EFF4FE491EEBD9898FC0187
:10013000EE5CFF4FE491EBBDFC01EA5BFF4FE49105
:10014000E9BDFC01E65AFF4F849188BD08950F93E5
:100150001F93CF93C82F8B01CC2359F085E0DCDFB0
:10016000C801B7DFB0DFC801B4DFC801B2DFC150DA
:10017000F3CFCF911F910F910895CF93DF93D82F95
:1001800064E170E08AE0E3DF84EF91E0A2DF8D2F8D
:1001900064E6A6D0CAE06C2FA3D0892F68EC70E08B
:1001A000D6DFA4DF8D2F6C2F9BD0D92F99D0892F2C
:1001B00068EC70E0CCDF9ADF68EC70E08D2FC7DF71
:1001C00095DF64E170E08AE0C2DF84EF91E0DF91C7
:1001D000CF917FCFC3981895989901C0C39A18956D
:1001E00018958FE384BBB99AB89ABC9ABB9A81E000
:1001F0008ABD83BF9AB590629ABD9AB590689ABD40
:100200009FEF9DBD80BF80E68CBD82E080BF80B740
:10021000806480BF89B7846489BF97B328B3892F6E
:1002200090E0809590958B7F822B88BBAA9AC2988C
:10023000AA9A8BB780628BBF8AB785608ABF85B761
:10024000806285BF789455DF8CE291E042DF5CDF0D
:1002500094DFFACF1124882009F01895F89416B885
:1002600032DFB998B898BC98BB9830E021E094E0B0
:1002700060E27EE486B38470222369F081112AC093
:1002800086E0881510F021E0F5CFCB010197F1F75A
:1002900020E099E0EFCF332319F0882321F01AC032
:1002A00031E0811130E085B7877E806185BF892F7D
:1002B000887011F440E401C040E6892F8770842BD8
:1002C00081BD85B7846885BF8B7F85BF789488950D
:1002D000F894D0CF8FE58DBF82E08EBF1FBE81DF47
:1002E000991B79E004C0991F961708F0961B881F88
:0C02F0007A95C9F780950895F894FFCF27
:00000001FF
